:1013D8005831252B352E326620205832252B352EB4
:1013E8003266005931252B352E3266202059322598
:1013F8002B352E3266005A31252B352E32662020A9
:101408005A32252B352E3266004531252B352E32A2
:101418006620204532252B352E32660047617573CC
:10142800736D65746572000418000001414443300F
:101438000000000001000404180000014144433189
:101448000000000001000804180000014144433274
:101458000000000001000C0418000001414443335F
:10146800000000000100100418000001414443344A
:101478000000000001001404180000014144433535
:101488000000000001001804180000014144433620
:101498000000000001001C0418000001414443370B
:1014A80000000000010020041800000144414330FE
:1014B80000000000010024041800000144414331E9
:1014C80000000000010028041800000144414332D4
:1014D8000000000001002C041800000144414333BF
:1014E80000000000010030041800000144414334AA
:1014F8000000000001003404180000014441433595
:10150800000000000100380418000001444143367F
:101518000000000001003C0418000001444143376A
:10152800000000000100400132000000556E6920F3
:10153800444143000100440132000000556E692017
:10154800414443000100450132000000322E355667
:101558002041444301004604180000094F41444318
:101568003000000001004704180000094F414443BF
:101578003100000001004B04180000094F414443AA
:101588003200000001004F04180000094F41444395
:101598003300000001005304180000094F41444380
:1015A8003400000001005704180000094F4144436B
:1015B8003500000001005B04180000094F41444356
:1015C8003600000001005F04180000094F41444341
:1015D80037000000010063045D00000947414443EF
:1015E80030000000010067045D00000947414443E2
:1015F8003100000001006B045D00000947414443CD
:101608003200000001006F045D00000947414443B7
:1016180033000000010073045D00000947414443A2
:1016280034000000010077045D000009474144438D
:101638003500000001007B045D0000094741444378
:101648003600000001007F045D0000094741444363
:101658003700000001008304180000094F4441438B
:101668003000000001008704180000094F4441437E
:101678003100000001008B04180000094F44414369
:101688003200000001008F04180000094F44414354
:101698003300000001009304180000094F4441433F
:1016A8003400000001009704180000094F4441432A
:1016B8003500000001009B04180000094F44414315
:1016C8003600000001009F04180000094F44414300
:1016D800370000000100A3045D00000947444143AE
:1016E800300000000100A7045D00000947444143A1
:1016F800310000000100AB045D000009474441438C
:10170800320000000100AF045D0000094744414376
:10171800330000000100B3045D0000094744414361
:10172800340000000100B7045D000009474441434C
:10173800350000000100BB045D0000094744414337
:10174800360000000100BF045D0000094744414322
:10175800370000000100C300000000000000000086
:10176800000000000000000405020301000706064F
:071778000700010203040554
:0D2E0C00019401011E0044000000000000C0
:101CAC00E4F5D4F5D7F5D175A4BD7580FF75A59D68
:101CBC007590FFEF6078E4F538E53825E025E024F1
:101CCC0024F582E43400F58312077B00000000E564
:101CDC003825E025E02487F582E43400F5831207EB
:101CEC007B00000000E53825E025E024A7F582E420
:101CFC003400F58312077B3F800000E53825E02592
:101D0C00E02447F582E43400F58312077B000000E1
:101D1C0000E53825E025E02467F582E43400F583FE
:101D2C0012077B3F8000000538E538B4088BD2855C
:101D3C00D2927D527F031229997D037F011229993A
:101D4C00E51E12299175E8807F647E00122D057FB7
:101D5C00047E00122D7CD3EF9400EE940840047F97
:101D6C000180027F00900045EFF07F027E00122D73
:101D7C007CD3EF9400EE940840047F0180027F0036
:101D8C00900046EFF0E4FFFE122D7CD3EF9400EEB2
:101D9C00940840047F0180027F00900044EFF0E43F
:101DAC00F5E87F10122C447F11122C44E4F538E531
:101DBC00382408FF122C440538E538C3940840EF4A
:011DCC0022F4
:102D7C0075D102E4F5BAEF540FF5BB75BCE0C2AFE8
:102D8C00C2EDD2EC30EDFDD2AF122627AFBFEFFE75
:042D9C00ADBEEDFFDC
:012DA0002210
:0325A300C9EFC9B4
:1025A600C283E4FF7E08C284E95ED394004003D36D
:1025B6008001C39287D284EEC313FE0FBF04E7E403
:1025C600FF7E08C284ED5ED394004003D38001C32E
:1025D6009287D284EEC313FE0FBF04E7CFEACFCDB6
:1025E600EFCDE4FF7E80C284ED5ED394004003D33A
:1025F6008001C39287D284EEC313FE0FBF08E7EBB8
:10260600FDE4FF7E80C284ED5ED394004003D38058
:1026160001C39287D284EEC313FE0FBF08E7D283AD
:012626002291
:0C19A400151FA81FEFF6E51F24FAF51F21
:1019B0002406F8E625E025E02487F582E43400F5E6
:1019C00083E0F8A3E0F9A3E0FAA3E0FBE8C0E0E5D8
:1019D0001F2406F8E625E025E02424F582E43400FF
:1019E000F583E0FCA3E0FDA3E0FEA3E0FFD0E0F878
:1019F000120029E51F2406F8E625E025E024A7F5D6
:101A000082E43400F583E0F8A3E0F9A3E0FAA3E070
:101A1000FB12011EA81F080812074A900044E0703C
:101A200003021AF2E4FFFEFDFCA81F080812071DBE
:101A30001202C45025E51F2406F8E625E025E0241F
:101A400024F582E43400F58312077B00000000A82F
:101A50001F080812076200000000900046E0704274
:101A6000FFFE7D207C41A81F080812071D1202C43A
:101A700060274025E51F2406F8E625E025E024241C
:101A8000F582E43400F58312077B41200000A81F93
:101A9000080812076241200000E4FBFA792078412F
:101AA0008041E4FFFE7D207C40A81F080812071D2E
:101AB0001202C460274025E51F2406F8E625E0252C
:101AC000E02424F582E43400F58312077B402000F3
:101AD00000A81F080812076240200000E4FBFA7902
:101AE000207840E8C0E0A81F0808120711D0E0F8ED
:101AF0008056E4FFFE7D207CC1A81F080812071D48
:101B00001202C4500BA81F0808120762C12000006F
:101B1000E4FFFE7D207C41A81F080812071D120269
:101B2000C4600D400BA81F08081207624120000086
:101B3000E4FFFE7D207C41A81F080812071D12004B
:101B40002DE4FBFA79A078411202277B007AFF7915
:101B50007F784712011EE4FBFAF9783F12002D123C
:101B6000036FA81FEEF608EFF6E51F2406F8E6540B
:101B70000790176F93F6FDA81FE6FA08E6FB7F03B0
:031B80001225A388
:071B8300E51F2407F51F22F6
:08299100C454F0440FFD7F0265
:10299900C294E4FEC293C297D2930EBE04F6E4FE3B
:1029A9007C08C293EF5CD394004003D38001C392A7
:1029B90097D293ECC313FC0EBE04E7D294C294E4FD
:1029C900FE7C80C293ED5CD394004003D38001C3A5
:0E29D9009297D293ECC313FC0EBE08E7D29483
:0129E70022CD
:062803008B5B8A5C895D1D
:10280900C294E4FEC293EEB40103D38001C392974C
:10281900D2930EBE04EEE4FE7D08C293EF5DD3941D
:10282900004003D38001C39297D293EDC313FD0EE9
:10283900BE04E7D294C294E4FE7D80AB5BAA5CA996
:102849005D1205D8C29330960DAB5BAA5CA95D12E7
:1028590005924D1205D8D293EDC313FD0EBE08E4BF
:02286900D29407
:01286B00224A
:0622B4008B3D8A3E893FCC
:1022BA00C294E4F540C293E540B40103D38001C35C
:1022CA009297D2930540E540B404EAE4F5407E08CB
:1022DA00C293EF5ED394004003D38001C39297D296
:1022EA0093EEC313FE0540E540B404E4D294C294CD
:1022FA00E4F540AB3DAA3EA93F1207AC000000003E
:10230A00AB3DAA3EA93F1206D778011206C41206AF
:10231A00F7C293AB3DAA3EA93FEBC0E0EAC0E0E9B1
:10232A00C0E012072AA296E4334BFFEAFEE9FDE871
:10233A00FCD0E0F9D0E0FAD0E0FB1206F7D2930520
:08234A0040E540B418BAD2943A
:012352002268
:101B8A00309503021CAB7B007A0079357F04122260
:101B9A00B4AF38AE37AD36AC35E4120331E4FBFAF4
:101BAA007980784B1202277B0A7AD77923784012F8
:101BBA00011E8F3C8E3B8D3A8C397F007E507DC34F
:101BCA007C47AB3CAA3BA93AA83912011EE4FBFAAE
:101BDA00F9783F12002D1221597B007A5079C37887
:101BEA00471202278F3C8E3B8D3A8C39900046E093
:101BFA007041900045E0600CE4FBFA797A78401273
:101C0A00011E80277B0A7AD779237840AF3CAE3B06
:101C1A00AD3AAC39120227E4FBFA79A078411201F5
:101C2A001EE4FBFA792078C112002D8F3C8E3B8D81
:101C3A003A8C39E51E25E025E02447F582E4340094
:101C4A00F583E0F8A3E0F9A3E0FAA3E0FBAF3CAE2A
:101C5A003BAD3AAC39120029E51E25E025E02467A0
:101C6A00F582E43400F583E0F8A3E0F9A3E0FAA3EF
:101C7A00E0FB12011E8F3C8E3B8D3A8C39C2AFE5D8
:101C8A001E25E025E02404F582E43400F5831207DA
:101C9A0056D2AFE51E045407F51E90177793122902
:011CAA0091A8
:011CAB002216
:102C4400151FA81FEFF6A81FE6FFD39407400CEF4B
:102C540094105007EF24F8FF1219A4A81FE6FFB43C
:102C64001008900044E024FF9290EFB41109900002
:0A2C740045E024FFB39282051F2201
:052E42008F2F7F00222C
:102CAE008B2F8A308931120592AB32AA33A9341296
:102CBE0005D8AB2FAA30A9319000011205ABAB326B
:0D2CCE00AA33A9349000011205EA7F02220A
:101FC200E4FDFF12000E7BFF7A1379D8900004E043
:101FD200FCA3E0FDA3E0FEA3E0F53B8E3A8D398C35
:101FE20038900014E0FCA3E0FDA3E0FEA3E0F53F7F
:101FF2008E3E8D3D8C3C120FCB7D01E4FF12000E14
:102002007BFF7A1379EB900008E0FCA3E0FDA3E0EC
:10201200FEA3E0F53B8E3A8D398C38900018E0FC37
:10202200A3E0FDA3E0FEA3E0F53F8E3E8D3D8C3C98
:10203200120FCB7D02E4FF12000E7BFF7A1379FEB2
:1020420090000CE0FCA3E0FDA3E0FEA3E0F53B8ED4
:102052003A8D398C3890001CE0FCA3E0FDA3E0FE31
:10206200A3E0F53F8E3E8D3D8C3C120FCB7D03E409
:10207200FF12000E7BFF7A147911900010E0FCA38E
:10208200E0FDA3E0FEA3E0F53B8E3A8D398C38905B
:102092000020E0FCA3E0FDA3E0FEA3E0F53F8E3EBE
:0720A2008D3D8C3C020FCBC9
:102C0600121B8A122E1DC8ECC8C9EDC9CAEECACB62
:102C1600EFCB900000E0FCA3E0FDA3E0FEA3E024E0
:102C260064FFE43EFEE43DFDE43CFCD31206B34003
:0D2C36000C122E1D900000120756121FC236
:012C4300226E
:102DC50020202020557067726164696E670020209D
:0E2DD50020204669726D776172652E2E2E00E9
:032E19000188002D
:10177F00E47888F675FFDE75FFAD75E104F5E27567
:10178F00E34075A401F5A5F5A675A72075B167759A
:10179F00B20875FF0775FFA5F5FE43B28075EF0818
:1017AF00122AE4E4F536F5377D01AF37122D2E05F9
:1017BF0037E53770020536C39401E536940040E8EB
:1017CF00E4F520C216C212C219C214D215C218C231
:1017DF00177888F6C2B57866F67864F618F6786AE0
:1017EF00F6F536F537746C2537F8E4F60537E53737
:1017FF00700205366414453670EBE4F536F5377430
:10180F00802537F8E4F60537E537700205366408AA
:10181F00453670EB122E4C7D08E4FF122DA11227D6
:10182F0096E47869F67861F67861E6FF75F010A4B2
:10183F00242FF582E5F03414F583E493FE786926BE
:10184F00F6EE600578610680DFEFD39400402A90B2
:10185F00143CE493FB740193FA740293F9745512D8
:10186F0005D812059264556002D21774AA1205D8D2
:10187F0012059264AA6002D2171220A9EF60030228
:10188F00196CC21574FFF508F509F50AF50BE4F5A7
:10189F000CF50DFE7F10FDFB7A00790E1207FC751B
:1018AF003BFF753C14753D24753E00753F107B0062
:1018BF007A00790E122A92E4F536F537E537C4F837
:1018CF00540FC868FFE536C454F048FE742F2FF547
:1018DF008274143EF583E493607C74332FF5827425
:1018EF00143EF583E49320E262E4F535E535C378E1
:1018FF0094965057E537C4F8540FC868FFE536C4BF
:10190F0054F048FE742F2FF58274143EF583E49340
:10191F00FD7C00C004C0057D00743C2FF58274145B
:10192F003EF583E493FB740193FA740293F978699B
:10193F00E68535F0A4FFE92FF9EA35F0FAD007D0A4
:10194F00061207FC122E4C053580A10537E53770BE
:10195F000205360218CB7F01121CAC8016D215E49B
:10196F00FF121CACE5EF30E30AD203050DE50D7055
:10197F0002050CE4F536F5377A007B967D03AF3719
:10198F001226AB0537E53770020536C39401E536ED
:04199F00940040E48C
:0119A3002221
:052E4700786AE6FF229D
:03002300021ED7E3
:101ED700C0E0C0F0C083C082C0D075D000C000C0D1
:101EE70001C002C003C004C005C006C0073099275F
:101EF700C2997864067964E778666670097864F64B
:061F0700D213C2B58011E7
:081F0D007524140000D524FB2B
:101F15007864E62480F8E6F599209803021FA72047
:101F25009A07201604C2988075C29A7863E606243B
:101F35006CF8A699C2987863E6FFB40113786CE64D
:101F4500FE70057863F6805AEE54072402786BF626
:101F5500EFB4020E786BE6B40908786DE6240379D0
:101F65006BF77863E6FFB4140476008035EFC37829
:101F75006B96402E7863E624FFFDE434FFFC7B007E
:101F85007A00796C12248B7863E6246BF8E66F602F
:031F950002800BBC
:081F98007524140000D524FBA0
:101FA00012090978637600D007D006D005D004D096
:101FB00003D002D001D000D0D0D082D083D0F0D0D6
:021FC000E0320D
:10272400786AE6FF18E68FF0A47C002527FFEC35D5
:10273400F0FE786DE675F010A4243CF582E5F034E3
:1027440014F583E493FB740193FA740293F98F8272
:0C2754008E831205ABFF7B007A00792514
:102760008F2F8B308A318932EA494B6016120592DD
:10277000FFE52FFD7C00120003AB30AA31A932EF38
:032780001205D867
:082783007533140000D533FB8F
:0B278B00852F993099FDC299022E4C59
:082DE3007866EFF6C213D2B5C9
:082DEB00752F140000D52FFB29
:062DF3007880E6F599224C
:102B7D00C9EFC9E964017028EDC39B40347894E630
:102B8D00FFEB2FFFE433FEEDC39FEE6480F87480FE
:102B9D0098501ED216C3ED9B786AF67865760122A1
:102BAD00B90214ED6B700AD216786AF67865760262
:082BBD0022C216E47865F6223D
:1028D000C9EFC9BAFF15BBFF12ED6B7002EC6A704D
:1028E00049D216786AF67865E9F622E9640170251E
:1028F000C3ED9BEC9A401C7894E62BFFE43AFEC3B0
:10290000ED9FEC9E500DD216C3ED9B786AF678656C
:102910007601228015B90218ED6B7002EC6A700A1C
:10292000D216786AF67865760222C216E47865F6E1
:012930002284
:10090900786CE6FF54F8F526EF1207D6094F090966
:100919005A0A09691009721109811209941909A859
:100929001A09C72009CC280A53290B03330B32377C
:100939000B55390B65410B6E490B77500BBB610B9E
:10094900B39800000BE6786DE6FDE509FB7F0180B1
:1009590021786DE6FC08E6FDAB09AA087F01802530
:10096900D21678657603020BE6786DE6FDE50BFB9A
:100979007F02122B7D020BE6786DE6FC08E6FDABE3
:100989000BAA0A7F021228D0020BE6786DE6FDE574
:1009990009FB7F01122B7D201603020BE6801678D6
:1009A9006DE6FC08E6FDAB09AA087F011228D020F4
:1009B9001603020BE6788076787F01020BE3D214E6
:1009C900020BE6C2ACE4F525D2B5FB7A0079257FA6
:1009D9007F1227607B007A0079257F181227607BB8
:1009E900007A0079257F031227607861E61227597A
:1009F9007B007A007925AF081227607B007A00799D
:100A090025AF091227607B007A007925AF0A1227E2
:100A1900607B007A007925AF0B1227607B007A0092
:100A29007925AF0C1227607B007A007925AF0D126A
:100A39002760E4F527740E2527F8E61227590527BC
:100A4900E527C3941040EE020AF1786DE6FFC378FA
:100A590061964003020BE675F010EFA4242FF5828E
:100A6900E5F03414AF82F52D8F2EC2ACE4F525D212
:100A7900B5FB7A0079257F7F1227607B007A0079A0
:100A8900257F0D122760852E82852D83E4931227F9
:100A990059852E82852D83740193122759852E82BB
:100AA900852D83740293122759852E82852D83748F
:100AB9000393122759852E82852D83740493122757
:100AC90059E4F527E52E2405F582E4352DF583E56E
:100AD900822527F582E43583F583E49312275905A6
:100AE90027E527C3940840DC7B007A007900AF250D
:100AF900122760C2B5D2AC020BE6786DE6FFB401ED
:100B09000B08E6F50808E6F509020BB3EFB402088D
:100B1900786EE6F508020BB3786DE6B4030808E6CB
:100B2900F50A08E6F50B020BB3E4F527E527C378C8
:100B39006D965016746E2527F8E6FF740E2527F872
:100B4900C6EFC60527E527B410E2805E7A007B323E
:100B59007D01786AE6FF1226AB020BE6786DE62482
:100B6900FF92028078786DE624FF9201806F786A9F
:100B7900E66005752902800B201805752903800395
:100B89007529017880767908A6297C007D027B0089
:100B99007A00798012248B7882EFF67F03122DE395
:100BA900E52964017037D2198002D212788876F16A
:100BB900802B7A007B327D017F001226AB7880760C
:100BC90079786DE67881F67C007D027B007A007980
:100BD9008012248B7882EFF67F03122DE3E52664D9
:100BE900A06003020D86786CE664A16003020CB76D
:100BF90008E6FFC37861964003020D8675F010EF91
:100C0900A4242FF582E5F03414F583E493F52975CE
:100C1900F010EFA42433F582E5F03414F583E4935E
:100C290030E22F122E428F297880767F08A629E597
:100C3900292402FDE433FC7B007A00798012248B9D
:100C490074822529F8EFF6E5292403FF122DE30222
:100C59000D86786DE6FF122E42C2ACE4F525D2B5B9
:100C6900E529D39406402C7B007A0079257F7F12F1
:100C790027607B007A007925AF29122760E4F527E0
:100C8900E527C395295007122724052780F205294E
:100C9900020D77E5292478122759E4F527E527C3BA
:100CA90095295007122724052780F2020D77786CC1
:100CB900E664A26003020D867861E6FF786DE6FEC0
:100CC900C39F4003020D8608E6FDC39F4003020D42
:100CD90086EEC39D4003020D8618E6F527E4F52943
:100CE900E527D3786E96501FAF27122E4275F01064
:100CF900E527A4242FF582E5F03414F583E4932540
:100D090029F529052780D9C2ACE4F525D2B5FB7AA6
:100D19000079257F7F1227607B007A007925AF292A
:100D2900122760786DE6F527E527D3786E96503E51
:100D3900E4F52875F010E527A4242FF582E5F034B1
:100D490014F583E493FFE528C39F501E786AE6FFF4
:100D590018E68FF0A47C002528FFEC35F0FE75F02D
:100D690010E52712273C052880C9052780BA7B0092
:100D79007A007900AF25122760C2B5D2ACE52664A6
:100D8900587047FA7B327D01786AE6FF1226AB7507
:100D990032007533007534817B007A00796D122C2D
:100DA900AE8F29E52924787880F6E5292401FDE428
:100DB90033FC7B007A00798012248B74812529F811
:100DC900EFF6E5292402FF122DE3E5266480600988
:100DD900E52664886003020F687865E6B4010F7A36
:100DE900007B327D01786AE6FF1226AB801AE4F5B2
:100DF90027E527C3789496500F7A007B327D01AF9F
:100E0900271226AB052780E9786CE65407F529B443
:100E1900070A75280108E6F529088005E4F5287808
:100E29006DE6F52A1529E52AC37861964003020F74
:100E39004675F010E52AA4242FF582E5F03414F55F
:100E490083E493FFE529D39F40028F297865E6B4AF
:100E59000109786AE6F52CF52B8009E4F52B7894DD
:100E6900E614F52C786AA62B786AE6D3952C40030C
:100E7900020F3AE4F527E527C395294003020F2F0E
:100E890075F010E52AA42433F582E5F03414F583CE
:100E9900E49330E203020F2A75F010E52AA4243006
:100EA900F582E5F03414F583E4936438701BE52981
:100EB900D394044008E5282527246E802A7863E620
:100EC900C39527FF746A2F801E75F010E52AA424A4
:100ED9002FF582E5F03414F583E493FFC37863E6D4
:100EE9009F25272528246BF8E6FD786AE6FF18E692
:100EF9008FF0A4FFE5277A002FFFEA35F0FE75F0A1
:100F090010E52AA4243CF582E5F03414F583E49332
:100F1900FB740193FA740293F98F828E83ED1205A3
:100F2900EA0527020E7FAF2A122C44786A06020EC0
:100F390071786AA62BE52664887024800FE52AB4A7
:100F4900FF1D786EE6F520E526B48813788076785B
:0F0F59007863E6246BF8E67881F67F02122DE3C9
:010F68002266
:107000007888E664F1600302747C3013FDC2AF75CA
:10701000FFDE75FFADE4F53FF53E209829E4F5432A
:10702000F54420981DC3E5449488E5439413501219
:0870300075490A0000D549FB77
:107038000544E54470E4054380E0B2B480D4859902
:107048003EC298E53E641A60030270F7F543F544C2
:0E70580020981DC3E5449488E543941350121C
:0870660075490A0000D549FB41
:10706E000544E54470E4054380E030989F85993FE0
:10707E00C298E4F543F54420981DC3E5449488E591
:05708E004394135012B1
:0870930075490A0000D549FB14
:10709B000544E54470E4054380E020980302701A30
:1070AB0085993FC298E4F543F54420981DC3E54408
:0870BB009488E5439413501280
:0870C30075490A0000D549FBE4
:1070CB000544E54470E4054380E020980302701A00
:0970DB0085993FC298D2B5C29913
:0870E4007549140000D549FBB9
:1070EC007599783099FDC2B502746EE53E640170F5
:0570FC0027D2B5C29986
:087101007549140000D549FB9B
:087109007599783099FDC299D7
:087111007549140000D549FB8B
:10711900E4F5993099FDC2B502746EE53E640260EA
:10712900030271C6F543F54420981DC3E5449488CC
:06713900E543941350121F
:08713F0075490A0000D549FB67
:107147000544E54470E4054380E020980302701A83
:1071570085993FC298E4F540E53F13B392B4E53F04
:1071670025E0FEC3E49400EE94705029E53F7F00CC
:1071770025E0FEC39460501DE5B654F04408F5B60B
:10718700758F038E458F468546828E83E4F053B60E
:0C719700F0F58F80037540FFD2B5C2995F
:0871A3007549140000D549FBF9
:0871AB007599783099FDC29935
:0871B3007549140000D549FBE9
:1071BB008540993099FDC2B502746EE53E6403605B
:1071CB00030272E7F543F54420981DC3E544948808
:0671DB00E543941350127D
:0871E10075490A0000D549FBC5
:1071E9000544E54470E4054380E020980302701AE1
:1071F90085993FC298E4F543F54420981DC3E544B9
:087209009488E5439413501230
:0872110075490A0000D549FB94
:107219000544E54470E4054380E020980302701AB0
:10722900859941C298E53F1392B4E53F25E0FEC335
:10723900E49400EE9470400302701AE53F7D002546
:10724900E0FCC39460400302701AE5B654F04408A8
:10725900F5B6758F01E54175F020A42DFFE5F03CE9
:10726900F5458F46E4F542E542C394205043E4F5E1
:1072790043F54420981DC3E5449488E5439413508D
:0172890012F2
:08728A0075490A0000D549FB1B
:107292000544E54470E4054380E020980302701A37
:1072A2000546E546AE457002054514F5828E83E536
:1072B20099F0C298054280B653B6F0E4F58FD2B584
:0272C200C2996F
:0872C4007549140000D549FBD7
:0872CC007599783099FDC29913
:0872D4007549140000D549FBC7
:1072DC00E4F5993099FDC2B502746EE53E64046024
:1072EC000302737BF543F54420981DC3E544948851
:0672FC00E543941350125B
:0873020075490A0000D549FBA2
:10730A000544E54470E4054380E020980302701ABE
:10731A0085993FC298E53F25E0F547754800E4F5B1
:10732A0040F543F5440548E548AE47700205471461
:10733A00F5828E83E4932540F5400544E5447002C6
:0E734A0005437004E543640270DBD2B5C299BE
:087358007549140000D549FB42
:087360007599783099FDC2997E
:087368007549140000D549FB32
:107370008540993099FDC2B502746EE53E640560A2
:1073800003027466F543F54420981DC3E5449488D0
:06739000E54394135012C6
:0873960075490A0000D549FB0E
:10739E000544E54470E4054380E020980302701A2A
:1073AE0085993FC298E4F543F54420981DC3E54402
:0873BE009488E543941350127A
:0873C60075490A0000D549FBDE
:1073CE000544E54470E4054380E020980302701AFA
:0973DE00859941C298D2B5C2990B
:0873E7007549140000D549FBB3
:0873EF0075997F3099FDC299E8
:0873F7007549140000D549FBA3
:1073FF007599203099FDE53F25E0FCE54175F020BA
:10740F00A42400FFE5F03CF5478F48E4F540F54232
:02741F00C29910
:087421007549140000D549FB78
:10742900854882854783E493F5993099FD0548E5B8
:1074390048AE477002054714F5828E83E4932540D0
:0B744900F5400542E542B420CDC29999
:087454007549140000D549FB45
:10745C008540993099FDC2B58008E53EB4060375A8
:10746C00EF10E53E6407600302701A7888F6D2AF1D
:01747C0022ED
:10262700122E4C20150B7A007B327D017F0012267B
:10263700AB30170B7A007B1E7D017F001226AB3073
:10264700121C3018197A007B327D01786AE6FF1276
:1026570026ABC212E4F50CF50D122209D21530197A
:102667002A301827C219122E2AE4FDFF12000E7B0A
:10267700FF7A2D79C5122CDB7D01E4FF12000E7B5A
:10268700FF7A2D79D3122CDB127000122E1DE47BFA
:102697002C7A01F9F8C31206B35002D2183014038A
:0426A70075EF102299
:0B2E370012177F122627122C0680F8CD
:101DCD00005EBCE2613FDD83C29C7E20A3FD1F410E
:101DDD009DC3217FFCA2401E5F01E3BD3E6082DCFE
:101DED00237D9FC1421CFEA0E1BF5D0380DE3C62EE
:101DFD00BEE0025CDF81633D7C22C09E1D43A1FFDE
:101E0D004618FAA427799BC584DA3866E5BB5907CD
:101E1D00DB856739BAE406581947A5FB7826C49ABD
:101E2D00653BD987045AB8E6A7F91B45C6987A24AD
:101E3D00F8A6441A99C7257B3A6486D85B05E7B99D
:101E4D008CD2306EEDB3510F4E10F2AC2F7193CD8D
:101E5D00114FADF3702ECC92D38D6F31B2EC0E507D
:101E6D00AFF1134DCE90722C6D33D18F0C52B0EE6D
:101E7D00326C8ED0530DEFB1F0AE4C1291CF2D735D
:101E8D00CA947628ABF517490856B4EA6937D58B4D
:101E9D005709EBB536688AD495CB2977F4AA48163D
:101EAD00E9B7550B88D6346A2B7597C94A14F6A82D
:101EBD00742AC896154BA9F7B6E80A54D7896B351D
:0A1ECD0070B8DCEEF4F7FAFDFEFF3A
:10248B00151F151FA81FECF608EDF6151F151F15C8
:10249B001FA81FC6EBC608C6EAC608C6E9C6E51FD5
:0424AB0024FCF51FF9
:1024AF00F80808E4F6A81FF608F6E51F2407F9A8B0
:1024BF001FE6FE08E6FFC3099719E76480F8EE648C
:1024CF0080985037E51F2404F8CBE6CB08E6FA08CE
:1024DF00E6F98F828E831205ABA81F080866FFE509
:1024EF001F2403F8EFF6E6901DCD93A81F0808F6FA
:1024FF00A81F0806E61870B20680AFA81F0808E6E6
:01250F00FFCC
:07251000E51F2409F51F225D
:07000300ED6F901DCD93FF8E
:01000A0022D3
:102DA100EF701E7598D0E589540F4420F58953C8FA
:102DB100E1438E10ED901ECC93F58DD28ED2ACC234
:032DC100BCD2AFD2
:012DC40022EC
:102AE400D2AFD2A9D2BBE589540F4401F589E4F5EC
:102AF4008E758CDBF58AD28CF55AF559F558F55755
:102B0400FFEF25E025E02490F8E4F6EF25E025E04A
:102B14002491F8E4F6EF25E025E02492F8E4F6EFBA
:0D2B240025E025E02493F8E4F60FBF01D46E
:012B31002281
:02235300151F54
:10235500A81FE4F6A81FE6FFC3940140030223ED7E
:10236500EF25E025E02493F8E6FFD394004052A83A
:102375001FE625E025E02491F8E67045EF30E015ED
:10238500A81FE6FF25E025E02493F8E6D394014055
:10239500047D0080067D01A81FE6FF122BC5A81F3E
:1023A500E6FF25E025E02493F816E66014EF25E026
:1023B50025E02492F8E6FEEF25E025E02491F8EEED
:1023C500F6A81FE625E025E02491F8E6600116A8A9
:1023D5001FE6FF25E025E02493F8E670057D011250
:0823E5002BC5A81F06022359B5
:0323ED00051F22A7
:03000B0002293196
:10293100C0E0C0F0C083C082C0D0E8C0E0E9C0E020
:10294100EAC0E0EBC0E0ECC0E0EDC0E0EEC0E0EFDB
:10295100C0E0758CDCE55A2401F55AE43559F55986
:10296100E43558F558E43557F557122353D0E0FFB5
:10297100D0E0FED0E0FDD0E0FCD0E0FBD0E0FAD02A
:10298100E0F9D0E0F8D0D0D082D083D0F0D0E032DE
:102D2E00151FA81FEDF6151FA81FEFF6A81FE6FF2B
:102D3E00C39401500D08E6FEEF25E025E02490F83F
:072D4E00EEF6051F051F2230
:1026AB00151F151FA81FEAF608EBF6151FA81FED3F
:1026BB00F6151FA81FEFF6A81FE6FFC39401505293
:1026CB00EF25E025E02493F8E67047A81FE6FB25ED
:1026DB00E025E02491F8E67039A81F08E625E00410
:1026EB00FFA81FE6FA25E025E02493F8EFF6A81FD4
:1026FB000808E6FE08E6FF7C007D0A12060CEA25B8
:10270B00E025E02492F8EFF6EB25E025E02491F8A4
:09271B00E4F6E51F2404F51F2279
:102BC500151FA81FEDF6151FA81FEFF6A81FE6FF96
:102BD500C39401501CEF25E025E02490F8E6601130
:102BE500A81F08E670047F0180027F00A81F08EF78
:102BF500F6A81FE6700608E624FF92B4051F051F18
:012C050022AC
:0C2E1D00C2AFAF5AAE59AD58AC57D2AF9F
:012E29002286
:042E4C0075FFA52247
:042D05008E3A8F3B38
:102D0900E4F53CF53DC3E53D953BE53C953A50146A
:102D19007FE87E0312287E122627053DE53D70E5F2
:042D2900053C80E104
:012D2D002283
:10286C0054F0FFE5A054014FF5A0A21192A37F01F3
:02287C007E00DC
:04287E008E538F5492
:10288200D3E55494FAE5539400500AEFD3940040F0
:102892003C001F80F6855355855456D3E55694FA6D
:1028A200E555940040157FFA7E0012287E740625B5
:1028B20056F55674FF3555F55580E0D3E55494002E
:0D28C200E55394004007AF56AE5512287E36
:0128CF0022E6
:0829E8008B3E8A3F89408D41BE
:1029F000122E4CAB42AA43A9441206422400FFE522
:102A0000F03460FE853E45853F46854047E4FDED58
:102A1000C39541501BEF2DF582E43EF583E493AB63
:102A200045AA46A9478D827583001205EA0D80DF0D
:0D2A3000AB42AA43A944E48541F002066DC3
:0823F0008B448A4589468D47A4
:1023F8007888E664F1600302248AC2AFE5B654F037
:102408004408F5B6758F01AB48AA49A94A12064295
:102418002400FFE5F034607889F608EFF6AA45A9AC
:1024280046788DA64408C6EAC608C6E9C6E4788B8D
:10243800F6788BE6C395475032788DCBE6CB080803
:1024480006E618CAE6CA70010614F9120592788CD5
:10245800F6E6FF78890806E618CCE6CC7001061483
:10246800F5828C83EFF0788B0680C6E4F58F53B63F
:10247800F0AB48AA49A94A8547F012066DD2AF12B7
:022488002E4CD8
:01248A00222F
:102A3D007888E664F1704DC2AFE5B654F04408F500
:102A4D00B6758F03788B7660087600E47889F60882
:102A5D00F6788BE6FE08E6F5828E83E4F0122E4CB6
:102A6D0026F618740236F61806E618700106C378B5
:102A7D008AE6940818E66480948040D5E4F58F5377
:042A8D00B6F0D2AF1E
:012A91002222
:10220900122A3DE4F542F543F548754900754A42FD
:10221900FB7A0079087D161223F0E4F53FE53FC308
:102229007894965067E4F53E75F010E53EA4242FA6
:10223900F582E5F03414F583E493604C7869E6851A
:102249003FF0A4FFAEF075F010E53EA4243CF58202
:10225900E5F03414F583E493FB740193FA74029363
:102269002FF9EA3EFA75F010E53EA4242FF582E530
:10227900F03414F583E493FD754800754900754AF7
:10228900421223F0053E80A0053F809175401275EA
:102299004134754800754900754A427B007A0079D6
:0A22A900407D021223F0E47888F66D
:0122B3002208
:1020A900E4F53CF53DF54275430075443CFB7A0087
:1020B90079087D161229E8E4F539E539C37894964B
:1020C9005067E4F53875F010E538A4242FF582E55A
:1020D900F03414F583E493604C7869E68539F0A40B
:1020E900FFAEF075F010E538A4243CF582E5F03434
:1020F90014F583E493FB740193FA7402932FF9EABC
:102109003EFA75F010E538A4242FF582E5F0341471
:10211900F583E493FD75420075430075443C12292B
:10212900E8053880A005398091754200754300752E
:10213900443C7B007A00793A7D021229E8E53B6448
:0F214900347004E53A641270047F0180027F0055
:012158002264
:102B32008F52301A4543A0F075A60FC2A3D2A2123B
:102B4200287AD2A17F0A7E0012287E20A7FDC2A188
:102B520012287AC2A275A6FF12287AE55212286CB0
:102B6200D2A112287AC2A112287AE552C412286C84
:0B2B7200D2A112287AC2A112287A22F8
:102C7E008F3A53A00FE53A54F042A0D2A112287A0F
:102C8E00C2A112287A53A00FE53AC454F042A0D242
:102C9E00A112287AC2A112287A7F647E0002287EB1
:10279600E4F538F53975A6FF53A00143A020D2A170
:1027A6007F01FE12287EC2A17F017E00122D057FC9
:1027B60020122C7E43A0F075A60FC2A3D2A2122827
:1027C6007AD2A17F647E0012287E30A703C21A2225
:1027D600D21AC2117F24122B32C2117F09122B3258
:1027E600C2117F20122B32C2117F0C122B32C21162
:0C27F6007F01122B32C2117F06122B3221
:0128020022B3
:0D2E2A00C2117F01122B32E4FDFF02000EE9
:10000E00ED5403C43354E0FEEF541F44804EFFC240
:04001E0011022B326E
:102DF9008F51C3E551648094A04005D211122B3242
:032E0900AF5122A4
:102D55008B5E8A5F8960AB5EAA5FA960120592608F
:102D6500150560E5607002055F14F9120592FFD242
:072D750011122B3280E02255
:100026000203DBE86480F8E933E83360110460F02A
:10003600ED33EC337009E8FCE9FDEAFEEBFF220440
:1000460060DED3EB9FEA9EE99DE8C2E78CF0C2F73B
:1000560095F0400CE8CCF8E9CDF9EACEFAEBCFFB07
:100066001203A685D0F05804700320D5B3E80470B7
:10007600075002B2D50203E592D5EC0460F7E4CC52
:10008600C0E0C398F8603B94186008400DD0E0FBD0
:100096000203BDE4FBFAC9FC8028E830E406E4C9A3
:1000A600FBE4CAFCE830E305E4C9CACBFCE8540724
:1000B6006010F8C3E913F9EA13FAEB13FBEC13FC2F
:1000C600D8F130F52FC3E49CFCEF9BFFEE9AFEEDD2
:1000D60099FDD0E0FBEF4E4D4C701222DB0302037C
:1000E600E2EC2CFCEF33FFEE33FEED33FDED30E7B3
:1000F600EB0203BDEF2BFFEE3AFEED39FDD0E0FB40
:1001060050130BBB00030203E5ED13FDEE13FEEFE8
:0801160013FFEC13FC0203BD12
:10011E00EC4D6011E8497017ED33EC3304600DE4DB
:10012E00FCFFFEFD22E933E8330470F80203DB1214
:10013E0003A658046009E4CC248150062850090215
:10014E0003E52840030203E2C0E0EB4A7044B980A5
:10015E0006D0E0FB0203D1EF4E701CBD8008EBFF12
:10016E00EAFEE9FD80EBE98DF0A4FEE5F002020760
:10017E00E9CDF9EAFEEBFFEF89F0A4FCE5F0CE89BC
:10018E00F0A42EFFE435F0CD89F0A42DFEE435F079
:10019E008067EF4E7005BD80D780C3EF8BF0A4ACA7
:1001AE00F0EE8BF0A42CFCE435F0F8EF8AF0A42CE2
:1001BE00E5F038FCE433CB8DF0A42CFCE5F03BF8F5
:1001CE00EE8AF0A42CFCE5F038F8E433CF89F0A4E5
:1001DE002CFCE5F038CF3400CE89F0A42FFFE5F0EB
:1001EE003EFEE433C98DF0A42EFEE5F039CD8AF043
:1001FE00A42FFFE5F03EFEE43DFD33D0E0FB5007BB
:10020E000BBB000F0203E5EC2CFCEF33FFEE33FECD
:06021E00ED33FD0203BDFB
:100224000203E5EC5D046005E8590470030203DB96
:100234001203A6580460F6EC4860F2EC7004FDFE6C
:10024400FF22C860DB2481C85009C39860025006AD
:100254000203E29850CAF582E9294B4A7005AB8241
:100264000203D175F0007C1A7880C3EF9BEE9AEDFF
:1002740099400DC3EF9BFFEE9AFEED99FDE842F025
:10028400DC23ACF0D0E0FFD0E0FED0E0FDAB822078
:10029400E7101BEB60BAEC2CFCEF33FFEE33FEED02
:1002A40033FD0203BDE803F830E705C0F075F00044
:1002B400EF2FFFEE33FEED33FD40B830E7C280AAE6
:1002C40074F8CC6480CCC86480C8F582046043C3ED
:1002D400EB9FF5F0EA9E42F0E99D42F0E89C45F080
:1002E40060305018E5825FFFE582F42B5582FB50A5
:1002F400210ABA001D09B90019088016E5825BFBC2
:10030400E582F42F5582FF50090EBE00050DBD0095
:10031400010CC3EB9FF5F0EA9E42F0E99D42F0E840
:0D0324009C45F06007CC4820E701B3EC22B7
:1003310075F020800E75F010800575F0087D007E47
:10034100007F003392D530D5031206A5EC3340105F
:10035100EF33FFEE33FEED33FDEC33FCD5F0ED2250
:0E036100E5F0247EA2D513CC92E7CDCEFF228C
:10036F00EDD2E7CD33EC3392D524814006E4FFFE86
:10037F00FDFC22FCE4CFCECDCC24E0501174FF80E5
:10038F00EDC3CC13CCCD13CDCE13CECF13CF047082
:07039F00F030D5DE0206A5D7
:100F6900E54C2438F8E6054C227835300F027838FC
:100F7900E475F0011207C60205922008EB7F2ED214
:100F8900088018EF540F2490D43440D4FF300C0B50
:100F9900EF24BFB41A0050032461FFE54D60021528
:100FA9004D0550E5507002054F300F0D7835E47549
:100FB900F0011207C6EF0205D8022DF97403D20F0A
:100FC9008003E4C20FF54C8B358A368937E4F54D39
:100FD900F54FF550E54D60077F20120FA480F57598
:100FE9004EFFC209C208C20AC20BC20DC20EC2100C
:100FF900120F72FF700D300F057F00120FB5AF5041
:10100900AE4F22B4255FC2D5C20C120F72FF24D095
:10101900B40A00501A75F00A784D30D50508B6FFA4
:101029000106C6A426F620D5047002D20B80D92465
:10103900CFB41A00EF5004C2E5D20C0212A2D209B1
:1010490080C6D20880C0D20A80BCD2D580BAD20D5F
:1010590080B47F20120FA4200A077401B54D004007
:10106900F1120F69FF120FA4020FDDD210D20E8008
:1010790095120F69FB120F69FA120F69F94A4B7041
:101089000679997A137BFF200A2EE54D602A7E00A6
:101099008E827583001205AB60060EEE654E70F008
:1010A900C2D5EBC0E0EAC0E0E9C0E0EE121302D01D
:1010B900E0F9D0E0FAD0E0FB120592FF60AAEBC09C
:1010C900E0EAC0E0E9C0E0120FA4D0E02401F9D0C1
:1010D900E03400FAD0E0FBE54E0460DCD54ED9805F
:1010E90087D20A80A21212E560F7E54E7001041258
:1010F90003F0A94E600DE54E600914F54E12138CEC
:10110900EF60F3EA30E702F404C3995077EAF42573
:101119004E0430E701E404F54E800D1212E560C17A
:10112900EA054E254E1203F0EA784BF630E701E462
:10113900254E04D54E04200D0114121302E4C0E01B
:1011490012138C784BE6601320E70714F6120F8C04
:10115900802204F6D0E014C0E07F00120F8CE54E27
:101169006007120F83154E800B300D03120F83D0C9
:10117900E0020FDDD0E00480C51212E560A0E54E63
:10118900041203F0784BEAF6E54E200D02600104E3
:05119900240412130202
:10119E0074FF04C0E012138C120F8CE54E200D026A
:1011AE006003120F83D0E0B54EE87F45120F96789C
:1011BE004BE67F2B30E7047F2DF404C0E0120FA422
:1011CE00D0E075F00A84C0F0120F8DD0E0120F8DB2
:1011DE00020FDD791080027908C20EC2108008D28B
:1011EE00D5790A8004790AC2D5E54E047002F54E0F
:1011FE00E4FAFDFEFF120F69FC7B08200913120FA3
:10120E0069FD7B1030080A120F69FE120F69FF7B11
:10121E0020EC3382D592D55013C3E43008069FFFDD
:10122E00E49EFEE42009039DFDE49CFCE4CBF8C2A1
:10123E0009EC700CCFCECDCCE824F8F870F3801703
:10124E00C3EF33FFEE33FEED33FDEC33FCEB33FB3C
:10125E00994002FB0FD8E9EB300905F8D0E0C448FD
:10126E00B209C0E00AEC4D4E4F78207B0070C2EA06
:10127E00B54E0040BCC0E0121304D0F0D0E02009FF
:10128E0004C4C0E0C4B209C0F0120F8DD0F0D5F086
:10129E00EB020FDD1207D6107A5311E158104B4CAA
:1012AE0010474211E54F11ED4411ED491060431105
:1012BE00F35511244611824510EE4713B950104FC5
:1012CE002D10532E10762B10572310742013A22A94
:1012DE00100F480000106EE54EB4FF03754E061257
:1012EE000F69FC120F69FD120F69FE120F69FF786C
:1012FE004402041F790AA2D5200B14300D09B9102F
:10130E00020404B9080104A2D5200E0250010420E3
:10131E000A68920AB54D005034C0E07F20300B1998
:10132E007F30A20A720E720D500F12135BC20AC2E8
:10133E000EC20DC2107F30800F300D03E9C0E012D7
:10134E000FA4300D03D0E0F9D0E0B54DCC300D1721
:10135E007F30B9100C120FA47F58300C077F7880A5
:10136E0003B90803120FA4300A057F2D020FA47FC4
:10137E00202010F87F2B200EF322920A80CF7F00C0
:10138E00B4070050052444F8E6FF22286E756C6CF5
:10139E002900D209120F693009F8C209784D30D5EB
:1013AE000108F602100F2D50434958120F692403FD
:1013BE00B405004001E49013B493120F95743A12E1
:0A13CE000F95D20B754D040211E1DA
:102159008F408E3F8D3E8C3D74FFFFFEFDFCAB40F2
:10216900AA3FA93EA83DC31206B3602C7F807E9684
:102179007D187C4BAB40AA3FA93EA83D1202C46022
:102189000250157F807E967D187CCBAB40AA3FA973
:102199003EA83D1202C45009AF40AE3FAD3EAC3D32
:1021A90022AF40AE3FAD3EAC3D12036F8F448E432C
:1021B9008D428C41EC120331C8ECC8C9EDC9CAEE95
:1021C900CACBEFCBAF40AE3FAD3EAC3D120029E4E8
:1021D900FBFAF9F81202C4601A401874FF2544F595
:1021E90044E54334FFF543E54234FFF542E5413424
:1021F900FFF541AF44AE43AD42AC41EC120331228D
:1003A600E9D2E7C933E833F892D5EDD2E7CD33EC9D
:0703B60033FC5002B2D52216
:1003BD00EC30E7100FBF000C0EBE00080DBD0004A1
:1003CD000BEB6014A2D5EB13FCED92E7FD2274FF4D
:1003DD00FCFDFEFF22E480F8A2D574FF13FC7D80A6
:0303ED00E480EFBA
:1003F000F920E72824F950037907E4F42402FB18D4
:10040000DBFDE624FB5014E9600DE4F618E604F683
:0F041000B40A08E4F6D9F57401F60A22C2D5221F
:10041F00ED33EC3392D5FA602AB4FF33EDC2E77BAC
:10042F00FF60067A047944E4227A04794D20D504DA
:10043F007A047948224E614E002B494E46002D49D1
:10044F004E4600E47A08F608DAFC7B00740722E8CF
:10045F00C0E0ECC0E0EDC0E0EEC0E0EFC0E0EA7558
:10046F00F010A4CAABF075F04DA42BFBE435F0FCF3
:10047F00EA2410FAEB34C5FBEC34D9FCEDC2E7FFEC
:10048F0075F056A4F42411C5F0F434C58FF0A42AE6
:10049F00E5F03BE43CF620E714120552D0E0FFD024
:1004AF00E0FED0E0FDD0E0FC1202278014F404122D
:1004BF000552D0E0FFD0E0FED0E0FDD0E0FC12010D
:1004CF001ED0E0F8E6FAEDD2E7CD33EC332482FB11
:1004DF00E4C3CF33CFCE33CECD33CD33DBF37B0776
:1004EF0075F00A846004F6081B0AE5F0F6088FF031
:1004FF00740AA4FFACF08EF0740AA42CFEACF0507A
:10050F00010C8DF0740AA42CFDE435F0F608DBDE47
:03051F007407223C
:100522003F8000004120000042C80000447A0000E1
:10053200461C400047C35000497424004B18968063
:100542004CBEBC205A0E1BCA6753C21C749DC5AE5A
:10055200FB60065407601C2323120580EB543860AD
:100562000912056C12057B12011EECF8EDF9EEFA88
:10057200EFCB22EB12057B80F1543803241C90054B
:1005820022FE93FC0EEE93FD0EEE930ECE93FF220F
:03000000022517BF
:0C251700787FE4F6D8FD75819402255E03
:10059200BB010689828A83E0225002E722BBFE0267
:0905A200E32289828A83E493229A
:1005AB00BB010CE58229F582E5833AF583E0225005
:1005BB0006E92582F8E622BBFE06E92582F8E2224F
:0D05CB00E58229F582E5833AF583E4932269
:1005D800BB010689828A83F0225002F722BBFE0102
:0205E800F322FC
:1005EA00F8BB010DE58229F582E5833AF583E8F047
:1005FA00225006E92582C8F622BBFE05E92582C8F3
:02060A00F222DA
:10060C00C2D5EC30E709B2D5E4C39DFDE49CFCEE09
:10061C0030E715B2D5E4C39FFFE49EFE120828C351
:10062C00E49DFDE49CFC800312082830D507C3E44C
:06063C009FFFE49EFE2278
:10064200BB010A89828A83E0F5F0A3E02250068783
:10065200F009E71922BBFE07E3F5F009E319228945
:0B066200828A83E493F5F07401932278
:10066D00BB010789828A8302087D500B09C5F027DB
:10067D00F7C5F01937F722BBFE0D09F8E325F0F3A6
:10068D00C5F019E338F322F889828A837401932522
:08069D00F0C5F0F8E4933822E7
:0E06A500C3E49FFFE49EFEE49DFDE49CFC2266
:1006B300EB9FF5F0EA9E42F0E99D42F0E89C45F09D
:0106C3002214
:1006C400E8600FEFC333FFEE33FEED33FDEC33FC94
:0306D400D8F12238
:1006D700BB010789828A830208935005E9F802075C
:1006E70011BBFE05E9F802089F89828A830208ABDD
:1006F700BB010789828A830207565005E9F802077A
:0A0707004ABBFE05E9F80208E422EF
:0C071100E6FC08E6FD08E6FE08E6FF2214
:0D071D00E6FB08E6F908E6FA08E6CBF8224C
:10072A00BB010789828A830208BB5005E9F80207E0
:10073A001DBBFE05E9F80208C789828A830208D42C
:0C074A00ECF608EDF608EEF608EFF622DB
:0C075600ECF0A3EDF0A3EEF0A3EFF02216
:10076200D083D082E493F608740193F6087402935E
:09077200F608740393F674047395
:10077B00A8828583F0D083D082120792120792123F
:10078B000792120792E473E493A3C583C5F0C58364
:10079B00C8C582C8F0A3C583C5F0C583C8C582C8C8
:0107AB00222B
:1007AC00BB010789828A8302077B5005E9F802079F
:0A07BC0062BBFE05E9F80208F02216
:1007C600FAE6FB0808E6F925F0F618E6CA3AF62234
:1007D600D083D082F8E4937012740193700DA3A3B2
:1007E60093F8740193F5828883E4737402936860C6
:0607F600EFA3A3A380DFC6
:102CDB00120592601CFF09E970010AC0E0EAC0E02E
:102CEB00EBC0E0122DF9D0E0FBD0E0FAD0E0F98098
:0A2CFB00DF7F0A122DF9E4FEFF222C
:102A92008B388A39893AE4F540F541E53F153FAE76
:102AA2003E7002153E4E6033AB3BAA3CA93D120577
:102AB20092FFAB38AA39A93A0541E541AC40700210
:102AC200054014F5828C83EF1205EAEF60CD7401A4
:102AD200253DF53DE4353CF53C80C0AB38AA39A92B
:022AE2003A2296
:1007FC00EF4E6012EF60010EEDBB010B89828A8314
:10080C00F0A3DFFCDEFA2289F05007F709DFFCA920
:0C081C00F022BBFEFCF309DFFCA9F02277
:10252300022E37E493A3F8E493A34003F68001F269
:1025330008DFF48029E493A3F85407240CC8C333B9
:10254300C4540F4420C8834004F456800146F6DF88
:10255300E4800B0102040810204080902E0CE47EDE
:10256300019360BCA3FF543F30E509541FFEE4937D
:10257300A360010ECF54C025E060A840B8E493A344
:10258300FAE493A3F8E493A3C8C582C8CAC583CA6F
:10259300F0A3C8C582C8CAC583CADFE9DEE780BE27
:012E1C0000B5
:10082800BC000BBE0029EF8DF084FFADF022E4CCB4
:10083800F875F008EF2FFFEE33FEEC33FCEE9DEC7D
:10084800984005FCEE9DFE0FD5F0E9E4CEFD22EDC3
:10085800F8F5F0EE8420D21CFEADF075F008EF2F0D
:10086800FFED33FD4007985006D5F0F222C398FDFE
:050878000FD5F0EA229B
:10087D00C5F0F8A3E028F0C5F0F8E5821582700206
:06088D001583E038F022A3
:0C089300E0FCA3E0FDA3E0FEA3E0FF22D8
:0C089F00E2FC08E2FD08E2FE08E2FF2295
:1008AB00E493FC740193FD740293FE740393FF2293
:0C08BB00E0F8A3E0F9A3E0FAA3E0FB22C0
:0D08C700E2FB08E2F908E2FA08E2CBF822B1
:1008D400E493F8740193F9740293FA740393FB227A
:0C08E400ECF208EDF208EEF208EFF22250
:1008F000D083D082E493F208740193F208740293D7
:09090000F208740393F27404730D
:00000001FF
